:100000008A110A120528000009000730990083169A
:100010000510851005118312BC30A0000230A1002C
:1000200089212F20AC012C08013C031C2B28AD0199
:100030002D083B3C031C2528BC30A0000230A10049
:1000400089210130AD07031C18281F3083050130BA
:10005000AC07031C13281F3083050C282E28051419
:100060005830A0000230A1008921AF203121AF20FB
:100070003121AF203F216C2031215B203121DF2055
:100080003121842031218D20312131217C203121E9
:1000900090203121F7203121C720312163203121E7
:1000A00068203121312184209030A0000130A1004E
:1000B0008921051008005521662108006621552177
:1000C000552155210800662155216621552108003A
:1000D000662155215521080055210800552155213B
:1000E0006621552108006621662155210800552109
:1000F000552155215521080055215521080055212C
:1001000066216621662108006621552166210800C6
:1001100055216621552155210800662166210800D8
:1001200066215521080066216621662108005521B7
:100130006621662155210800662166215521662128
:1001400008005521662155210800552155215521CA
:100150000800662108005521552166210800552117
:100160005521552166210800552166216621080088
:1001700066215521552166210800662155216621F9
:100180006621080066216621552155210800662157
:1001900066216621662166210800552166216621B7
:1001A00066216621080055215521662166216621B8
:1001B0000800552155215521662166210800552149
:1001C00055215521552166210800552155215521DC
:1001D00055215521080066215521552155215521CC
:1001E0000800662166215521552155210800662108
:1001F0006621662155215521080066216621662168
:100200006621552108005521662155216621552179
:100210006621080066216621552155216621662147
:1002200008005521552166216621552155210800D8
:100230006621552155216621552108006621552149
:10024000552155216621080066215521552155214A
:1002500055216621080005115030A000A101892117
:10026000080005115030A000A10189215030A000E4
:10027000A10189215030A000A101892108000511A8
:100280005030A000A10189215030A000A101892196
:100290005030A000A10189215030A000A101892186
:1002A0005030A000A1018921080005150530840007
:1002B0000230AA009930A0000230A1003530A2001F
:1002C0000030A300C42105112B21080005150530BD
:1002D00084000230AA009930A0000230A100D23080
:1002E000A2000030A300C42105112B210800051530
:1002F000053084000230AA009930A0000230A1002D
:10030000EE30A2000230A300C42105112B21080009
:100310008829A008031994299B21A003000000004C
:100320000000000000008929A108031908009B2192
:10033000A103A00389290C30A500A50B9D2900006D
:1003400000001230A200A20BAA29AC21AC210000AF
:1003500000000800AC21A3290D30A400A40BAE2995
:10036000000008001030A8020001031C013EA90291
:10037000031C0800BB290A30A8020001031C013E2F
:10038000A902031C0800BB292A0880042008A80031
:100390002108A900B2210130A202031CA3032A09EB
:1003A00080052008A8002108A900B221A208031D89
:0A03B000C429A308031DC429080096
:02400E00C431BB
:00000001FF
